:020000040000FA
:06000000673002303A28CF
:08000800A000030EA100831209
:1000100081018B100B11210E8300A00E200E090010
:0C007400203084008001840A80300402E7
:10008000031C3C281230B000482183160C30850533
:1000900087018312850187010730990000309A009B
:1000A000103083168E008312603083168F00831207
:1000B0000030831691009F008312C83083168100A0
:1000C000831231309000003083168C008312103080
:1000D0008B00BC1B6D28851DD121782181018E01EB
:1000E0008F010B118B100B108C018B178A2031198B
:1000F0008C202A21B30B8828031085190314B90D0D
:10010000F03039020319D0210F3039020319C92107
:10011000F721762864000800080031110130B7008B
:100120008B132030370783169B001C141A08831288
:10013000A4001030370783169B001C141A08831282
:10014000A3000030370783169B001C141A08831283
:10015000A2008B17321CB22822090339A200A3097E
:10016000A409A50901303702031DBB283D18BB288F
:100170003D143E146C2102303702031DC428BD1803
:10018000C428BD143E146F2103303702031DCD284F
:100190003D19CD283D153E14722104303702031D50
:1001A000D628BD19D628BD153E147521B70A0530CD
:1001B00037020318080090280130B600B300B400DD
:1001C000B500B70085018701B1138A20B30B02295E
:1001D000031085190314B90DF030390203192029D1
:1001E000B41F8501B41F8701B40B02293708B60874
:1001F0000319B60003190029FF3085008700B603F4
:100200009630B400311DE5283111321C0C292D091E
:100210000339AD00AE09AF098B1320303707BB009F
:100220002F08BA00332110303707BB002E08BA0060
:10023000332100303707BB002D08BA0033218B175C
:1002400085018701B70AB60105303702031CE5288E
:10025000782108003E1C08003E101030BB003D080D
:10026000BA00332108008B133A0883161C159A0034
:1002700083123B0883169B0055309D00AA309D00D9
:100280009C1464009C1841291C1183128B170800D0
:10029000831600309B001C141A088312BC008316BE
:1002A00010309B001C141A088312BD0083162030E6
:1002B0009B001C141A088312C10041080F39C200A8
:1002C000410E0F39C3000130C2080319C2000130CA
:1002D000C3080319C30008000130BD000800023044
:1002E000BD0008000430BD0008000830BD00080053
:1002F000BD013D1401303D0203198D2902303D023C
:1003000003199C2904303D020319AB2908303D0232
:100310000319BA290130BD003E145830D30005122C
:100320008512051485108714071107148712071604
:1003300087110A30D40008004230D300051285121C
:1003400005108510871007110710871207128711F3
:100350000130D40008000530D300051285120514C1
:1003600085148710071107108716071687110A30A2
:10037000D40008000F30D300051685120510851033
:100380008710071507148712071287150A30D40043
:1003900008003E140310BD0D3D1A3D143D12782196
:1003A0000800B601B301B4013C1CD929BC01BC143E
:1003B000DB29BC013C143C08B6006400DF29E029BD
:1003C000E129E229E3293130B41B8500B41F8501FE
:1003D000B30BDD29B40BDD290310B60CB608031DE1
:1003E000DD290030BB003C08BA0033210800851D20
:1003F000023085190130BD008F08031908008E01F5
:100400008F01D0080319732AD00F082AEA23732A10
:10041000501C420850184308D107031C122AFF3011
:10042000D100EA2356180516D61885165619051454
:10043000D6198514561A8714D61A07155718071493
:10044000D718871657190716D719871551080E029E
:100450000318422A58180512D81885125819051081
:10046000D8198510581A8710D81A0711591807106B
:10047000D918871259190712D9198711FF3050025C
:10048000031908008F08031D08008A2051080E0276
:10049000031C422A56180512D61885125619051043
:1004A000D6198510561A8710D61A07115718071033
:1004B000D718871257190712D71987115818051618
:1004C000D818851658190514D8198514581A871480
:1004D000D81A071559180714D91887165919071665
:1004E000D91987150800D50B08004630D500D40B64
:1004F00008000130D000D10001305302031D872ACB
:10050000D61558160F30D4000230D3000800023040
:100510005302031D922AD71459140A30D400033011
:10052000D300080003305302031D9C2AD614053063
:10053000D4000430D300080004305302031DB52A50
:1005400056155814D81460308B1383169B001C1456
:100550001A0883128B173D190130D400043084002F
:100560000530BC184730D300080047305302031D44
:10057000C32A3D19D0013D190800D9140130D40017
:100580004830D300080048305302031DCF2AD71447
:100590000130D4000530840B4730D300080005300B
:1005A0005302031DF12A0130D400BC18E62A3D197C
:1005B000D0013D19D1013D1908005714D9140A3052
:1005C000D4000630BD184430D30008005714D914A5
:1005D0000A30D4004930BD184430D30004308400C0
:1005E000080049305302031DFB2A58150130D4007E
:1005F0004A30D30008004A305302031D072B56151A
:100600000130D4000630840B4930D3000800063096
:100610005302031D122BD61458150530D4000B308D
:10062000D30008000B305302031D1D2B5614D814A1
:100630000A30D4000C30D30008000C305302031DE4
:10064000282BD71559150A30D4000D30D3000800D7
:100650000D305302031D322B56160530D4000E30D8
:10066000D30008000E305302031D4B2BD616D815AD
:10067000581670308B1383169B001C141A088312B3
:100680008B17BD190130D400043084000F30BC1822
:100690004B30D30008004B305302031D592BBD19BA
:1006A000D001BD190800D9150130D4004C30D30059
:1006B00008004C305302031D652BD7150130D400C0
:1006C0000F30840B4B30D30008000F305302031D52
:1006D000832B0130D400BC187A2BBD19D001BD1971
:1006E000D101BD1908005715D9150A30D4001030B2
:1006F000D30008005715D9150A30D4004D30D30067
:100700000430840008004D305302031D8D2BD81691
:100710000130D4004E30D30008004E305302031D88
:10072000992BD6160130D4001030840B4D30D300F5
:10073000080010305302031DA42B5616D81605309E
:10074000D4000130D300080042305302031DB02B07
:10075000BC18D61456160130D4004330D30008001C
:1007600043305302031DBE2BBC18D8145816013059
:10077000D4004230BD1C4530D30008004430530241
:10078000031DCB2B5815D815591459150130D40019
:100790004230D300080045305302031DD82B5615B4
:1007A0005616571457150A30D4005830D300080095
:1007B00058305302031DE72BD61558161430D400B9
:1007C000043084000630BC184930D30008000130E2
:1007D000D300080056180516D618851656190514A4
:1007E000D6198514561A8714D61A071557180714E0
:1007F000D718871657190716D7198715D601D701A5
:1008000058180512D818851258190510D8198510CE
:10081000581A8710D81A071159180710D9188712B3
:0E08200059190712D9198711D801D9010800FA
:084000000600030005000500A5
:02400E00CC33B1
:104200000100FF00FF00FF00FF00FF00FF00FF00B4
:10421000FF00FF00FF00FF00FF00FF00FF00FF00A6
:104220000100FF00FF00FF00FF00FF00FF00FF0094
:10423000FF00FF00FF00FF00FF00FF00FF00FF0086
:104240002200FF00FF00FF00FF00FF00FF00FF0053
:10425000FF00FF00FF00FF00FF00FF00FF00050060
:10426000FF00FF00FF00FF00FF00FF00FF00FF0056
:10427000FF00FF00FF00FF00FF00FF00FF00FF0046
:10428000FF00FF00FF00FF00FF00FF00FF00FF0036
:10429000FF00FF00FF00FF00FF00FF00FF00FF0026
:1042A000FF00FF00FF00FF00FF00FF00FF00FF0016
:1042B000FF00FF00FF00FF00FF00FF00FF00FF0006
:1042C0003200FF00FF00FF00FF00FF00FF00FF00C3
:1042D000FF00FF00FF00FF00FF00FF00FF00FF00E6
:1042E0003200FF00FF00FF00FF00FF00FF00FF00A3
:1042F000FF00FF00FF00FF00FF00FF00FF000000C5
:00000001FF
